:030000000219FDE5
:03000B000200AA46
:03002B0002015F70
:03005B000202E7B7
:030073000202CDB9
:1000800002030406080C10182030406080040608A3
:100090000C10182030406080A0C000070F1F3F0DDB
:1000A0000D04050D050205030302C2AFC0D0C0E078
:1000B000206217E5256002E473E525F4F58A758B67
:1000C00000D262D0E0D0D0D2AF3285268AC262E5BB
:1000D00026F4602F758B00D0E0D0D0C293C295C2B9
:1000E00097D2AF32C293C295C297206E0C20660998
:1000F000740ED5E0FDE57E4290758B00D0E0D0D047
:10010000D2AF32758A00C28DD26201F901B930686E
:1001100005206602D29301B9306805206602D295A7
:1001200001B9306805206602D29701B9C2923068E1
:100130000A206607740CD5E0FDD29301B9C2943051
:10014000680A206607740CD5E0FDD29501B9C29605
:1001500030680A206607740CD5E0FDD29701B9C259
:10016000AFC2AD53E6EFC0D0C0E0D2D3D2AFC2CE63
:10017000E52A6007207449152A21C07800790020FB
:10018000742EE580307E01F430E30278FF53DACF3D
:10019000207E0343DA20307E0343DA10C2D8C271D6
:1001A000E580307E01F430E30279FFC3E89970CB3B
:1001B000306103752A18207403752A18885FD2707D
:1001C00020740DE52B6004152B21D043DA01C2D831
:1001D000207002412EA85F206102C270207436791F
:1001E00082B70431C3E894F0400374F0F8E8C454D3
:1001F0000F28F87984B703024115C313C31387216D
:10020000200802C313200A06C3C898F8411528F82D
:10021000500374FFF88822E52D54066011E533C3BE
:1002200013C31324062522F52250037522FF78827A
:10023000B6044E852224A824C3E52495644002A870
:1002400064C3E895664002A8668825E569700241A6
:100250007FC3E8AA699A5003E8FAE4F9EAC333FBDA
:10026000E56BF45B29400D256AF8E56A6002156AC2
:10027000400B417F0AC3E56A9A5002056A78FF88FD
:1002800026C3E52594404002D26420CF0AD0E0D0B6
:10029000D043E610D2AD32C2CF053A7801E52A60EC
:1002A00005307402152AC3E55F94014005756200AC
:1002B00041C3756300756C00E5622401F56250036B
:1002C0007562FFD0E0D0D043E610D2AD32C2AFC0ED
:1002D000D053E67FC2607591008556948557957519
:1002E0009104D0D0D2AF32C2AF53E6EFC2ADC0D08E
:1002F000C0E0C0F0D2D3D2AFA8FBA9FCC2D8307105
:1003000002614E53DACF207E0343DA10307E03437E
:10031000DA20D271E580307E01F420E30261258885
:10032000278928A17B53DACF207E0343DA20307E51
:100330000343DA10C2D8C271307402A1677800E5B5
:1003400080307E01F430E302A167885FA14F53DA69
:10035000CF207E0343DA20307E0343DA10C27120BF
:100360006102812753DACF207E0343DA10307E0307
:1003700043DA20C2D8D271885A895BC3E89558F80D
:10038000E99559F97B007E087A00C3E8948CE994DA
:10039000005005755E008119882178A2E6A82160C9
:1003A00055C3E894C8E994005008E4D2E4FB7A0A03
:1003B00061F4C3E89468E994015008E4D2E3FB7A5D
:1003C0000F61F4C3E894D0E994025008E4D2E2FB50
:1003D0007A1E61F4C3E894A0E994055008E4D2E1E0
:1003E000FB7A3C61F4C3E89498E994085008E4D29D
:1003F000E0FB7A787E00C3E8955CFCE9955DFD3012
:10040000E70AECF42401FCEDF43400FD755E00C352
:10041000EC9AED9E5003755E01885C895D855A58A3
:10042000855B597802A14FC3E89527F8E99528F92B
:10043000307C02A133307B02A133307A02A12C2020
:100440007502814AE9FDE8FC8169E9C313F9E81303
:10045000F8307902A12CE9C313F9E813F8307802D7
:10046000A12CE9C313FDE813FC20612CC3EC941C00
:0E047000ED940240028180ED701EC3EC94C832
:10047E0050180529E52970021529C3E529940A505B
:10048E0002A167755F00D270A167E5296002152988
:10049E007888E6F97400207F087896B90302789E72
:1004AE00E624FAFEE43400FFC3EC9EFCED9FFD92C1
:1004BE0008B90310A2085007207609D27681D230EF
:1004CE007602C276A2085016B9030DECF42401FC94
:1004DE00EDF43400FD0204EC78007900A133B90389
:1004EE0015EC33FCED33FDC3EC940AFCED9400FDEA
:1004FE0050047C007D00C3EC94FFED940040067820
:10050E00FF7900A133EC8575F0A4C5F0A2F733F89E
:10051E007900400302054F78FF790002054FE9C3C9
:10052E0013F9E813F8307C0EE9600278FFC3E81384
:10053E0038F8E43400F9C3E894FFE99400400278F7
:10054E00FF885FD270206102A167741FF4552F4B94
:10055E00F52FC274EB7002D274752A1830740375BD
:10056E002A0A306102A17B20740353DAFE20740341
:10057E00752B06D0F0D0E0D0D0D2AD43E610327954
:10058E00010205AB79030205AB790A0205AB791EB0
:10059E000205AB79640205AB79C80205AB7817E4A6
:1005AE00D5E0FDD8FAD9F6227A147B780205D27AF4
:1005BE00107B8C0205D27A0D7BB40205D27A0B7BAE
:1005CE00C80205D27902B27DE4C294D5E0FDD2957F
:1005DE00D5E0FDC295D5E0FDD294D5E0FDD293E5F0
:1005EE0076D5E0FDC2937496D5E0FDD9D9EAF8D55B
:1005FE00E0FDD8FBDBCEC29422C37C007D0075F0FB
:10060E000005F0EA33FAEB33FB50F6EB13FBEA137B
:10061E00FAC3E9FFE8FEE89AF8E99BF95004EFF90E
:10062E00EEF8B3EC33FCED33FDD5F0DFEDF9ECF87D
:10063E0022E889F08A20D2D4F8A9F07B0030F70B9B
:10064E007BFFF42401F8E9F43400F9E88520F0A4E6
:10065E00ADF0F8E98520F0A4AFF0FEED2EF97400B0
:10066E003FFA7C04C3EA13FAE913F9E813F8DCF451
:10067E008BF030F70AE8F42401F8E9F43400F9E8D5
:10068E0089F0C2D4F8A9F0227882B604030206F1EA
:10069E00C3E55F940140030206BB852224E4F545C1
:1006AE00F546F547F548F549C26D0206F17882E642
:1006BE00FCD26DE522F523783879C7AA40AB41C349
:1006CE00EB13FBEA13FAEC146013C3EB13FBEA1300
:1006DE00FAEC14146007C3EB13FBEA13FAD1078884
:1006EE0045894622C3E5459523F8E5469400F95021
:1006FE000CC3E89480E994FF4016020722C3E894E5
:10070E007FE994005003020722787F7900020722C6
:10071E00788079FF884A894B22E54A2547F8E54BD0
:10072E003548F9854B20E4300701F43549FA30E7B6
:10073E0009C3EA94F04015020760C3EA940F500310
:10074E0002076078FF79FF7A0F0207607800790060
:10075E007AF0C3E5249564500AC374019524500BB6
:10076E0002077EE54B20E70E02077EE54B30E706DB
:10077E00884789488A492278A4E6FAC3E54A33F8BD
:10078E00E54B33F9D13FE930E70BC3E89480E994A8
:10079E00FF4013E1B8C3E8947FE994005002E1B83A
:1007AE00787F7900E1B8788079FFE820E715C3E516
:1007BE002398F84009C3E8940140030207DF78014B
:1007CE000207DFE8F424012523F840030207DF784F
:1007DE00FF884C2278A5E6FAA848A949D13FE9300E
:1007EE00E70CC3E89401E994FF4016020813C3E82E
:1007FE0094FFE99400500302081378FF7900020871
:10080E0013780179FFE920E715C3E54C98F8400904
:10081E00C3E89401400302083A780102083AE8F46A
:10082E002401254CF8400302083A78FF88242278E8
:10083E00FFC26420693D206A12D264C3E541940A66
:10084E004009C3E52594405002C26479A1E76023B4
:10085E00E541601F74FF8541F0848539F0306A03ED
:0F086E0075F005A4F8C5F0600278FFC3E8956740
:10087D005002A867886622C3E5409440E541940183
:10088D00E5665003140195046002F5662202089D89
:10089D002275E890227883E6FFE5E820ECF7A8BD05
:1008AD00A9BE0573C3E57394084052757300E9FA48
:1008BD0079A0E76044EA7007E574601B0208D8C3AD
:1008CD00E895746010E5745006600C140208E40499
:1008DD0060F90208E4E574F574C394A8401B7564CF
:1008ED00C0C394054013756480C39405400B7564B3
:1008FD0040C39405400375640075BB0122E5642473
:10090D0010500274FFF5647982B704022131C3A837
:10091D0064E524985002A824C3E895664002A866B1
:10092D0088258826E573B4070375BB1E22743279BA
:10093D00A687F0A4C5F0A2F733F8C3E8956440028A
:10094D00A864882288248825882688672275400017
:10095D007541F022C2AF75C820A8CCA9CDAA3A30F6
:10096D00CF010A75C824D2AFAB3BAC3C883B893C68
:10097D00C3E89BF8E99C206908F9306702417621AC
:10098D00D3AD3D8A3DF9EA9DFA600478FF79FFAE5B
:10099D003EAF3F8B3E8C3FC3EC9FFCC3E99CF542C1
:1009AD00A83BA93CC3E89EF8E99FF9C3E54113FBB9
:1009BD00E54013FAE82AF540E93BF541500675404C
:1009CD00FF7541FF411DAA40AB41AC40AD417E04D6
:1009DD007F02C3EB940440021E1FC3EB9408400238
:1009ED001E1FC3ED13FDEC13FCDEF7C3EA9CFAEBFF
:1009FD009DFBEF6009C3E913F9E813F8DFF7EA2867
:100A0D00FAEB39FB8A408B4150067BFF8B408B41C3
:100A1D00C3EB94025002D2673069047F03414878DA
:100A2D0092E6FFC3E537948240110FC3E53794A0DA
:100A3D0040010FC3EF940640027F057E06E541C4D9
:100A4D00540FF9E541C454F0F8E540C4540F28F8AB
:100A5D00C3E89EFAE99400FB4009C3EA9402EB94C3
:100A6D000050047A02E4FB41C2AA40AB41EBC4FE44
:100A7D00EAC4540F4EFCC3EA9CFAEB9400FBC3E8A6
:100A8D0013C313F8EA28FAEB3400FB8A408B41C3F9
:100A9D00EB94024002C2677806EBC4FE7B00EAC409
:100AAD00540F4EFAC3EA98FA4005C3940250027AE5
:100ABD00027892E6FF30600241C285525685535747
:100ACD00D26043E680C3E49AF8E49BF93067026193
:100ADD005CE8FAE9FBD3E913FDE813FC885289536E
:100AED00C3EF94036038EF20E00DE82CF8E93DF9F1
:100AFD00ECFAEDFB020B17E828F8E939F9C3E82405
:100B0D0002F8E93400F97AFE7BFFC3EF9403400E3F
:100B1D008A548B55884E894F8C508D5161908854D5
:100B2D0089558A4E8B4F8C508D51306920C3E533DA
:100B3D0094034019E542A2E713F8E555F424013872
:100B4D00400B20E7087554FFF42401F5556190E83A
:100B5D00FAD3E813FC8852C3EF94036020EF20E032
:100B6D0007E82CF8ECFA617CE8282402F87AFEC339
:100B7D00EF940340088A54884E8C50619088548AB3
:100B8D004E8C50E56BC3335002646BF56B306002D5
:100B9D00619A753402D26043E680E52D54066026D5
:100BAD00A840A941C3E913F9E813F8C2AF53E67F92
:100BBD00759100C3E498F594E499F595759104D277
:100BCD006043E680D2AF22D26575440075200030B7
:100BDD006B03752040020BF3D26575440075204000
:100BED00306B03752000D2AF7801206722E52D54BC
:100BFD00066002C265C3E541940540137802940571
:100C0D0040087803940540027806306902780A207E
:100C1D006019E544601530690AC3E5339403400358
:100C2D00D53406D2AFD26C81CD71A2D2AF0000C245
:100C3D00AF206726E541C3FB940F40027B0FEB24E9
:100C4D000530730123306A02742820620123F930C4
:100C5D0069027982E58BC39940B50544E59E70051F
:0E0C6D00E59B020C74E59A5440B5200281B755
:100C7B0030690A08C3E8940A400108811C20650208
:100C8B0061F3C26553E67F75910030671075940070
:100C9B007595FE759104D26043E68061F3AE40AF6B
:100CAB0041C3E49EF594E49FF595819EC3E533948F
:100CBB0002500261F330650261F3D80281CB811CD3
:100CCB00C26C53E67F75910085549485559575914B
:100CDB0004854E56854F57D26043E680D2AFE52D43
:100CEB0054066008206A020533020D07306C0D2094
:100CFB006B0A206507158115810215972278003044
:100D0B0064053065027801E53775F007A4F9E5F065
:100D1B0028F5F0E9A2F013A2F113A2F213F537C3F1
:100D2B0094785003753778C3E53795384008D26609
:100D3B00C293C295C297306002A14185505685512E
:100D4B0057D26043E68022207D14C2AF754302C2A6
:100D5B0094D292D2AF759F33759E00020F33C2AF00
:100D6B00754302C294D296D2AF759F33759E000223
:100D7B000F33307243207D20C2AF75430390013D8A
:100D8B00757E10C297C296306204D295A19BD29405
:100D9B00D2AF759E23020F33C2AF75430390013D53
:100DAB00757E10C293C292306204D295A1BBD294CD
:100DBB00D2AF759E22020F33207D17C2AF7543034E
:100DCB00900118C297306202D295D2AF759E230262
:100DDB000F33C2AF754303900118C293306202D236
:100DEB0095D2AF759E22020F33207D11C2AF754392
:100DFB0004C292D296D2AF759E22020F33C2AF7548
:100E0B004304C296D292D2AF759E23020F33307237
:100E1B0049207D23C2AF75430590012C757E04C21A
:100E2B0095C294306204D293C137D292D2AF759FE0
:100E3B0033759E00020F33C2AF75430590014E759B
:100E4B007E40C295C294306204D297C15AD296D2D8
:100E5B00AF759F33759E00020F33207D1AC2AF759D
:100E6B00430590010EC295306202D293D2AF759FAB
:100E7B0033759E00020F33C2AF754305900122C23A
:100E8B00953062E8D297D2AF759F33759E00020FF3
:100E9B0033207D11C2AF754306C296D294D2AF7583
:100EAB009E23020F33C2AF754306C292D294D2AFC8
:100EBB00759E22020F33307242207D20C2AF7543E4
:100ECB000190014E757E40C293C292306204D2975C
:100EDB00C1DFD296D2AF759E22020F33C2AF7543DC
:100EEB000190012C757E04C297C296306204D29396
:100EFB00C1FFD292D2AF759E23E133207D16C2AFD4
:100F0B00754301900122C293306202D297D2AF7522
:100F1B009E22E133C2AF75430190010EC29730623E
:100F2B0002D293D2AF759E23C2662290010C757EBE
:100F3B0000C293C295C297C292C294C296C2622259
:100F4B00788076090876090876040876FF08760318
:100F5B000876FF087607087601087601087601788F
:100F6B008C76010876FF0876FF0876FF0876FF0877
:100F7B0076FF0876030876FF0876FF0876FF08767B
:100F8B00250876D00876280876500876040876FF70
:100F9B0008760208760008767A0876FF087601084C
:100FAB007601087600087603227887E6FFC272780E
:100FBB0088E6C394036008C27DE630E102D27DC2AD
:100FCB007E7889E630E102D27EC3EF940260087529
:100FDB008E01D273020FE7758E00C273227880E602
:100FEB00149000809378A4F67881E6149000809397
:100FFB0078A5F67886E61490008D9378A6F6789C03
:10100B00E67538FF75390CB402067538A075390AC8
:10101B00B4030675388275390578A3E61490009AE7
:10102B0093F569120F3622227896E6FA7897E6FB4B
:10103B007888E6B40305C3EB940EFB307F047A008B
:10104B007BFFC3EB9AFCC3948250027C82757500C4
:10105B000575EC8575F0A4C3E5F0947D40F222D2C2
:0F106B007F113312059C7A007B007C10120592D6
:10107A00E55F2AFA74003BFBDCF37C04C3EB13FB49
:10108A00EA13FADCF7FEC27F113322E5EF20E6030A
:10109A007520000520903DFFE520146006901FFF93
:1010AA001460009304600375EF1253D9BF7581C0B1
:1010BA0043FF8012058D75EF0243B203E5B32404A2
:1010CA0020E70DF521E5B120E0068521B343B10102
:1010DA00120F367580FF75A40075F1FE75D4F77589
:1010EA00900275A5FC75F2FC75D50075A0FD75A674
:1010FA000275F30275D60075B0FF75A70175F4FF86
:10110A0075E241E4F8F6D8FD756B01120F4B121522
:10111A00D978988676753001C2AF1205A61205B63F
:10112A0012059C1205BD12059C1205C412059CC22B
:10113A00AF78FA79FA308307D9FBD8F7021C001284
:10114A000FB4120FE81132113378988676120F36DF
:10115A0075885075891275C82475910475D84075BB
:10116A00A82275B80275E690759B80759D00759AE0
:10117A0080759C0075D10E75BC5875BB0175BA1F78
:10118A0075E88012058DD2AF12089A53DACF207E05
:10119A000343DA20307E0343DA1043DA01C2D8C2AD
:1011AA00711205A6D2617B037A0CE55E70077A0C90
:1011BA00DB0302113912059C207003021139C27037
:1011CA00E55FC3940240E1E52F541F856160F56134
:1011DA00B560D5DAD5C26153DACF207E0343DA206F
:1011EA00307E0343DA10C2D8C27178A2E67008D200
:1011FA0074E52F54E0F52FC2757529001205A13048
:10120A007409C3E529940A4002D27512059278023C
:10121A003074027800C3E55F9840F0C2AF1205B699
:10122A001205B61205B6D2AF1205A6754D0078881A
:10123A00E6B403026116120592788CE6C394015053
:10124A0003021316E530C3940150030213162074E7
:10125A0035C3E55F94FF5003021316C2AF1205CBE4
:10126A00D2AF1205A1C3E55F940150EFC2AF1205D8
:10127A00B61205971205B6D2AF1205A1C3E55F945F
:10128A00FF40E90217817F02D27F11331205A1C202
:10129A00AFC27F1133AE5FC3E55F947FD2AF4076B2
:1012AA0012058DC2AF1205CBD2AFDFDC116AC3EED5
:1012BA0094057897F61205A612161B1217047F0AD0
:1012CA00D27F11331205A1C2AFC27F1133AE5FC301
:1012DA00E55F947FD2AF50E612058DC2AF1205B614
:1012EA001205971205B6D2AFDFD6116AEE24057839
:1012FA0096F61205A612161B1217331205A1113300
:10130A00C3E55F94FF50024158021781C3E55F9518
:10131A004D4003855F4D1205A178017988E7B40332
:10132A00027805C3E55F9840024138C2AF1205CB87
:10133A001205CB1205CBD2AF1205A6753000E4F523
:10134A0031F5320531E531F470390532789AE678AB
:10135A0019146012783214600D787D14600878FAD6
:10136A00146003753200C3E532984017153275319F
:10137A00B478998676C2AF1205CBD2AF78988676C2
:10138A001205A1120597E52A7005307402213978F1
:10139A00012074027806C3E55F9840A77888E6C3FF
:1013AA00940360031205A1E52A7003021139C2AF42
:1013BA00120F36E4F522F523F524F525F526F56A0C
:1013CA00D2AF7885E6C333F568E4F545F546F547C7
:1013DA00F548F549F573F52CF52DF537757308754C
:1013EA00BB1E12058D12089EE5E820ECFBA8BDA9DC
:1013FA00BEE97001F888741208A275730875BB1EDD
:10140A007887E6FE7602120FB47887EEF6C2AF75D9
:10141A0064FF12093A852264852265852266D2AF65
:10142A0075220175240175250175260185636C7580
:10143A006D017888E6B40307C27D307602D27DD288
:10144A0068D269753300120E9C120EC112095A1223
:10145A00096112095A12096112095A021475C2AFB6
:0E146A00120FB4D2AF75730075BB01120BE503
:10147800120696120D08120D52120961120BD43081
:101488006D031206F220670312083D306703120845
:1014980084120D08120D7D120961120BE5306D03DF
:1014A800120727120D08120DF4120961120BD4301D
:1014B8006D03120785120D08120E19120961120B1D
:1014C800E5306D031207E2120D08120E9C12096135
:1014D80012089E120BD4120D08120EC11208A21285
:1014E8000961306935206B32856764856765856376
:1014F8006C756D0179187A0CC3E53399400FC26990
:10150800D26A8A35856764856766021522C3E55FF6
:101518009401400302147502159F306A1B206B1852
:10152800E535147004C26A8168F535C3E55F940136
:10153800400302147502159F753600C3E56278FAF8
:10154800985054307404E52A604D7888E6B403173F
:10155800207D05207607A16F307602A16F206B07EA
:10156800D26B85676481B478F0306B0585676478E1
:1015780020C3E5419850028175306B1BC26BC27D58
:10158800307602D27DD26A75351285676481750519
:1015980036E55F6002A1A2753600C2AF120F367839
:1015A80087E6FE7602120FB47887EEF6E4F522F5A8
:1015B80023F524F525F526F568C268D2AF12058D06
:1015C800120F36307409C3E536940540022139619B
:1015D80048901A0D782012165DE520B4550CA31218
:1015E800165DE520B4AA030215FB120F4B12161B59
:1015F80002161A901A0378807B0A12165DA308DB7C
:10160800F9901A0F788C7B1812165DA308DBF990F5
:101618001A2722C2AF12169C121676901A00740E60
:10162800121662A37404121662A37414121662903E
:101638001A0378807B0A121661A308DBF9901A0F47
:10164800788C7B18121661A308DBF91216AF1216F4
:101658008D901A2722E493F622E6438F01538FFDDB
:1016680075EF0275B7A575B7F1F0538FFE22438F5A
:1016780002438F0175EF0275B7A575B7F1901A0D82
:10168800F0538FFC22901A0D7455D162901A0E7483
:10169800AAD162227A3079D07820901A40D15DE5BB
:1016A80020F709A3DAF7227A3079D0901A40E7D1E7
:1016B8006209A3DAF922AB77A878BB01027980BB6B
:1016C80002027981BB03027982BB04027984BB05DB
:1016D800027986BB06027992BB07027987BB0802AA
:1016E80079A3BB0902799CBB0A027988BB0B0279F2
:1016F80089E8F7227C051205A6DCFB22C2AF120599
:10170800B61205BD1205C41205CB1205971205B60F
:101718001205BD1205C41205CB1205971205B612A3
:1017280005BD1205C41205CBD2AF22C2AF1205CB3C
:101738001205C41205BD1205B61205971205CB1283
:1017480005C41205BD1205B61205971205CB120580
:10175800C41205BD1205B6D2AF22AE77AF78C2AFBC
:101768001205B61205B61205B6120597DEF2120575
:10177800CB120597DFF8D2AF22F104D1FCD1FC756A
:101788007701757801757900F1627C05AD5F120506
:10179800A6C3ED955F70F5C3E55F9401400AC3E504
:1017A8005F94FF40320217BDD1BED11BF104C2AF16
:1017B80075EF12D1FCDCD50579C3E57994035002A5
:1017C80080C6D1FC0578E5771490009F93F808C38C
:1017D800E57898500280AED1FCD1FC0577C3E57757
:1017E800940C5002809C120F4BD11BC2AF75EF12A4
:0217F800D1FC22
:0319FD0002109540
:101A00000E0414090904FF03FF0701010155AA018F
:101A1000FFFFFFFFFF03FFFFFF25D0285004FF0259
:081A2000007AFF01010003FF41
:101A4000235467794B4631323041485623202020B9
:101A500023424C48454C4923463331302320202033
:101A60002020202020202020202020202020202076
:101C0000C2AFC2D353D9BF7581C043B20343FF8073
:101C1000752438752503B1C975EF0275E24043F1AB
:101C20000853A4F775D400D2837DFA780379E67C53
:101C300010752200752300901DD67B0675249875BB
:101C400025013083028142208308D8FBD9F9DCF7D3
:101C500081B4308308D8FBD9F9DCF781B4B189E4C9
:101C600093A3C39A6004DDC381B4DBDBB17B600264
:101C7000812B7B08E493FAA3B15CDBF87A30B15C8A
:101C8000752200752300B17BEAFCEBFDC3ED94FEE9
:101C9000400EB17B8A278B28ED30E0048A828B834B
:101CA000B17B7AC270D8C3ED94FE601350CEBD00F4
:101CB00025EC60097520007521FF0200008100A855
:101CC00027A9280809D804D90281D3B17FEA89AAB3
:101CD000F281C50D81A0C3ED94035049EDA2E092BD
:101CE000007AC5C3E5829400E583941C50902000DF
:101CF00010438F02438F0175B7A575B7F1F030001F
:101D00001FA827A9280809438F01538FFDD804D99C
:101D100002A12089AAE275B7A575B7F1F0A3A10DBC
:101D2000538FFC817C7AC1BD030CE493A3FAB140CC
:101D3000DCF8B138817C817EAA22AB23B15CEBFA5E
:101D4000EA6222752608C3E52313F523E52213F57D
:101D50002250066323A0632201D526EAB1C9B1C986
:101D600075260AEAF4200102D283300102C283B14F
:101D7000C9C3134002C201D526EB22B17FEAFB2082
:101D80008302A17F308302A184752608AE24AF258B
:101D9000C3EF13FFEE13FEB1CDB1C9C3EA13308315
:101DA000024480FA30E703632201C3E52313F523DD
:101DB000E52213F52250066323A0632201D526D91C
:101DC000E52265236523F52222AE24AF250E0FDE22
:101DD000FEDFFCD20122424C48656C693437316326
:041DE000F3100601F5
:00000001FF
